:020000000130CD
:02000B0041733F
:10003000758902D2A9D2AF758C06758A0075816F59
:10004000D2B9D28C7590FF75B0FF75300075310054
:10005000C209C211E5266422705BE541643870551F
:10006000300B2CE53245334534453554F07046208D
:100070001011201226853236853337853438853580
:1000800039019B85323D85333E85343F853540853A
:100090003632853733853834853935D208C20AC2BD
:1000A0000BC21051DEB20D200D2DC2AF7590FF7541
:1000B000B0FF438702753600753700753803753910
:1000C00000753D00753E00753F01754000D2137507
:1000D0002622754138018FC20BC210C2123009FDB1
:1000E0005107315D200A05D54202D2B7300A02110C
:1000F000F301DD20084C300A49E532653D702DE5FD
:1001000033653E7027E534653F7021E53565407005
:100110001BE53D453E453F45407004C2B78026C2C1
:10012000AFC20D7590FF75B0FF438702E5345401EF
:100130007010E5325401700A7403C395324003C253
:10014000B722D2B72275420F8536328537338538CC
:1001500034853935D208C20AC20BC21022A2B2823B
:10016000B3500A753C07753A01753B1022D20BD289
:10017000B7C208C20AC20DD53CF2753C07D53AECAD
:10018000853B3A153BE53BB40102053BA2B2B3B057
:10019000B3405B201105D211D21222C212A2B2507A
:1001A00024E53564097007E5346409700122E5250A
:1001B000B4320241F0753200B4330241FA753300B3
:1001C000B434EA6104E53220100464017009453357
:1001D00045344535700122E525B4320241B9753206
:1001E00000B4330241C3753300B434EA41CDC212C6
:1001F000D211201005D210C21322201305D210D222
:100200001322C210C213220520C209712D74035596
:1002100020F5202432F8E6301307301004740F80E4
:1002200005300E02241090025393300F0274FF43E6
:10023000B033F590E5207003C2B422147006201686
:1002400011C2B522147006201508C2B12220140272
:10025000C2B02214B78C85274544970405FFFFFFE1
:10026000FFFFEF10B38881234140930001FBFBFBAC
:10027000FBFBFFC0E0C0D005307414B530366230EF
:10028000D20905317464B5312B6231B20C200B24D4
:10029000300C21300A0451F041B4300817E5321413
:1002A000453445334535700A51B9C208D20AD210D7
:1002B00041B451B9D0D0D0E0321532E532F4701EDD
:1002C0007532091533E533F470147533051534E5CB
:1002D00034F4700A7534091535E535F47000752568
:1002E00034E535700A752533E534700375253222FF
:1002F0000532740AB5322475320005337406B533FD
:100300001A7533000534740AB53410753400053598
:10031000740AB53506753509753409752534E53522
:10032000700A752533E534700375253222C216C272
:1003300015C214E535700ED214E5347008D215E5F7
:10034000337002D216E520C20EB4020BD20E300872
:1003500006A20C820E920E300A05A20C920F2230D9
:0B036000B30630B2032010F2C20F22DF
